:060000000201B6020ECB66
:03000B0002094B9C
:03001300020AA43A
:01001B0032B2
:03002300020F5C6D
:01002B0032A2
:030033000206DBE7
:03003B000210B1FF
:01004300328A
:01004B003282
:01005300327A
:01005B003272
:01006300326A
:03006B000207C4C5
:030073000207DCA5
:03007B000207F287
:0300830002080868
:03008B0002082048
:03009300020862FE
:03009B000208ACAC
:0300A3000208ADA3
:0300AB000208AE9A
:0300B3000208AF91
:0300BB000208B088
:0300C3000208B17F
:0300CB000208B276
:0300D3000208B36D
:0300DB000208B464
:0300E3000208B55B
:0300EB000208B652
:0300F3000208B749
:0300FB000208B840
:030103000208B936
:03010B000208BA2D
:030113000208BB24
:03011B000208BC1B
:030123000208BD12
:03012B000208BE09
:030133000208BF00
:03013B000208C0F7
:030143000208C1EE
:03014B000208C2E5
:030153000208C3DC
:03015B000208C4D3
:030163000208C5CA
:03016B000208C6C1
:030173000208C7B8
:03017B000208C8AF
:030183000208C9A6
:03018B000208CA9D
:030193000208CB94
:03019B000208CC8B
:0301A3000208CD82
:0301AB000208CE79
:0301B3000208CF70
:030234000202378C
:0502370012023C80FEF4
:05023C00C203C201C273
:0402410002C20012E3
:0402450006DF750853
:030249000E750926
:03024C0012750A1E
:03024F0020750B0C
:0302520012750C16
:030255002A750DFA
:0302580012750E0E
:03025B004A750FD2
:03025E0012751402
:030261006A7515A6
:04026400127A0E7488
:0902680012FB54C0700302032BC9
:04027100751A0E7577
:030275001B127CDD
:040278008C7D127EE9
:0A027C000E7F12ECC39EFCED9FFD07
:0A02860074022CFCE43DFD8C168D83
:05029000177518007550
:0A0295001900780079007A007B0060
:09029F00C3E89516E99517EA95EC
:0A02A80018EB95195029748028FC0A
:0A02B200E439FDAE1AAF1BE82EF58B
:0E02BC0082E93FF583E0FE8C828D83F008B866
:0D02CA0000D309B900CF0ABA00CB0B80C8E1
:0702D700750880E4F5097AC7
:0A02DE000E7B12EA2480FAEB34FFD5
:0802E800FBE50AC39AF50AE5E3
:0502F0000B9BF50BE57E
:0602F50010C39AF510E5AC
:0502FB00119BF511E567
:0603000012C39AF512E59C
:05030600139BF513E557
:06030B000CC39AF50CE59D
:050311000D9BF50DE558
:060316000EC39AF50EE58E
:05031C000F9BF50FE549
:0603210014C39AF514E577
:04032700159BF51518
:0E032B00D2E843D82090E65CE0FA443DF0D2E0
:0C033900AF90E680E0FA20E105D204124B
:0203450012F3B1
:0C03470090E680E0FA54F7F0538EF8C204
:0103530003A6
:07035400120737300005120B
:04035B00039DC2003C
:09035F003003F212073850EDC220
:010368000391
:0C03690012143620012090E682E0FA30E9
:0A037500E70890E682E0FA20E1EAD2
:0E037F0090E682E0FA30E60890E682E0FA208E
:02038D00E0DAB4
:0A038F0012149512073CE43380BB02
:040399007582012246
:0C039D0090E6B9E0FA24F450030206C513
:0703A900EA2A2A9003B07359
:0703B0000204B7020562021E
:0603B70006C50206240247
:0603BD0006C50206C502A0
:0603C30003D40206C5028E
:0603C90004AF0204A702CC
:0503CF00049702049FE9
:0803D40012074040030206D2AB
:0A03DC0090E6BBE0FABA01028017B8
:0503E600BA020280488C
:0503EB00BA0302806767
:0503F000BA0602801AAC
:0503F500BA0702804B75
:0303FA0002048C6E
:0A03FD0090E6B3E509F0AA087B00C2
:0804070090E6B4EAF00206D20F
:0C040F00120399E582601290E6B3E50B41
:0B041B00F0AA0A7B0090E6B4EAF002B1
:0204260006D2FC
:0B04280090E6A0E0FA4401F00206D2CA
:0A04330090E6B3E511F0AA107B007B
:08043D0090E6B4EAF00206D2D9
:0A04450090E6B3E513F0AA127B0065
:08044F0090E6B4EAF00206D2C7
:0E04570090E6BAE0FAF5821213FFAA82AB8398
:0E0465007C008A058B068C07EA4B4C600F90DA
:0E047300E6B3EEF07E0090E6B4EDF00206D2A5
:0B04810090E6A0E0FA4401F00206D271
:0B048C0090E6A0E0FA4401F00206D266
:0804970012076DE4330206D2E6
:08049F00120763E4330206D2E8
:0804A700120744E4330206D2FF
:0804AF0012074EE4330206D2ED
:0804B70012078240030206D285
:0A04BF0090E6B8E0FABA8002800D62
:0504C900BA8102802D44
:0504CE00BA8202803E2D
:0304D300020557C8
:0A04D600E4A2013325E0FAE4A202DB
:0E04E00033FB420290E740EAF090E741E4F07F
:0D04EE0090E68AF090E68B7402F00206D2D0
:0E04FB0090E740E4F090E741F090E68AF09040
:08050900E68B7402F00206D239
:0E05110090E6BCE0FA53027E90E6BCE0FBC32D
:0E051F0074809BE433FB4A9014FD93FA3395ED
:0E052D00E0FB74A12AFA74E63BFB8A828B8302
:0E053B00E0FA53020190E740EAF090E741E455
:0E054900F090E68AF090E68B7402F00206D283
:0B05570090E6A0E0FA4401F00206D29A
:0805620012078640030206D2D5
:0C056A0090E6B8E0FA6008BA0202801BBC
:030576000206D2A8
:0B05790090E6BAE0FABA0105C20102E8
:0205840006D29D
:0B05860090E6A0E0FA4401F00206D26B
:0905910090E6BAE06003020619CD
:0E059A0090E6BCE0FA53027E90E6BCE0FBC3A4
:0E05A80074809BE433FB4A9014FD93FA339564
:0E05B600E0FB74A12AFA74E63BFB90E6BCE081
:0E05C400FC53047E90E6BCE0FDC374809DE411
:0E05D20033FD4C9014FD93FC3395E0FD74A1B5
:0E05E0002CFC74E63DFD8C828D83E0FC530400
:0E05EE00FE8A828B83ECF090E6BCE05480FA2B
:0E05FC00C423541FFA90E6BCE0FB740F5B9022
:0D060A00E6832AF090E683E0FA4420F00237
:0206170006D209
:0B06190090E6A0E0FA4401F00206D2D7
:0806240012078A40030206D20E
:0C062C0090E6B8E0FA6008BA02028026EE
:030638000206BBFC
:0B063B0090E6BAE0FABA0105D2010215
:0206460006D2DA
:0B06480090E6BAE0FABA02030206D204
:0B06530090E6A0E0FA4401F00206D29D
:0E065E0090E6BCE0FA53027E90E6BCE0FBC3DF
:0E066C0074809BE433FB4A9014FD93FA33959F
:0E067A00E0FB74A12AFA74E63BFB90E6BCE0BC
:0E068800FC53047E90E6BCE0FDC374809DE44C
:0E06960033FD4C9014FD93FC3395E0FD74A1F0
:0E06A4002CFC74E63DFD8C828D83E0FC43044B
:0906B200018A828B83ECF08017B1
:0A06BB0090E6A0E0FA4401F0800D83
:0D06C50012078E500890E6A0E0FA4401F004
:0906D20090E6A0E0FA4480F02259
:0406DB0053D8EF32CF
:0A14FD0000010202030304040505C8
:0E06DF0090E600E0FA74E75A90E6004410F04E
:0E06ED0090E601E0FA4440F090E61074A0F0B0
:0E06FB0090E61174A0F000000090E61274E288
:0E070900F000000090E61374E0F00000009095
:0E071700E6147422F000000090E6157420F045
:0A07250043AF011208D012114C126C
:06072F000A0112092C0270
:020735000E2F85
:01073700229F
:0407380075820122A3
:04073C00758201229F
:04074000758201229B
:0A07440090E6BAE0F51C7582012270
:0C074E0090E740E51CF090E68AE4F09093
:09075A00E68B7401F075820122A6
:0A07630090E6BAE0F51D7582012250
:0C076D0090E740E51DF090E68AE4F09073
:09077900E68B7401F07582012287
:040782007582012259
:040786007582012255
:04078A007582012251
:0A078E0090E6B9E0FABAD002800547
:05079800BAD12180121E
:0E079D0090E604E0FA43028000000090E604BB
:0407AB00EAF08011DF
:0D07AF0090E604E0FA547FF00000008004A2
:0407BC00758201221F
:0407C000758200221C
:0C07C400C0E0C082C083D2005391EF90CF
:0C07D000E65D7401F0D083D082D0E032EE
:0E07DC00C0E0C082C0835391EF90E65D7402CE
:0807EA00F0D083D082D0E03290
:0E07F200C0E0C082C0835391EF90E65D7404B6
:08080000F0D083D082D0E03279
:0C080800C0E0C082C083D2035391EF9087
:0C081400E65D7408F0D083D082D0E032A2
:0C082000C0E0C082C083C002C003850E8F
:03082C0010850F25
:04082F0011AA10AB4F
:0A083300118A828B83A37402F08502
:03083D000C128515
:030840000D13AAEB
:0A08430012AB138A828B83A37407A3
:0E084D00F05391EF90E65D7410F0D003D002EE
:07085B00D083D082D0E0320F
:0E086200C0E0C082C083C002C00390E680E008
:08087000FA30E724850C108525
:030878000D11AAB5
:0A087B0010AB118A828B83A3740274
:05088500F0850E128554
:03088A000F13AA9F
:0A088D0012AB138A828B83A3740759
:01089700F070
:0E0898005391EF90E65D7420F0D003D002D0B3
:0608A60083D082D0E03295
:0108AC003219
:0108AD003218
:0108AE003217
:0108AF003216
:0108B0003215
:0108B1003214
:0108B2003213
:0108B3003212
:0108B4003211
:0108B5003210
:0108B600320F
:0108B700320E
:0108B800320D
:0108B900320C
:0108BA00320B
:0108BB00320A
:0108BC003209
:0108BD003208
:0108BE003207
:0108BF003206
:0108C0003205
:0108C1003204
:0108C2003203
:0108C3003202
:0108C4003201
:0108C5003200
:0108C60032FF
:0108C70032FE
:0108C80032FD
:0108C90032FC
:0108CA0032FB
:0108CB0032FA
:0108CC0032F9
:0108CD0032F8
:0108CE0032F7
:0108CF0032F6
:0C08D00090E670E0FA543FF043B2C02202
:0408DC0043804022F3
:0408E0005380BF2260
:0808E400E58030E6030208E0A4
:0308EC000208DC23
:0408EF0043808022A0
:0408F30053807F228D
:0808F700E58030E7030208F37D
:0308FF000208EFFD
:07020F00E4F527F528E4F5F2
:0402160023F524F5B3
:03021A0025F526A1
:0A090200E521258AFA8A8AC3EA95E6
:0A090C0021500974012522258CF505
:020916008C2231
:07091800E522258CF58C227D
:0B091F00AA82AB838A047D008C218B30
:02092A00222287
:0E092C00C28C538EF75389F0438901758A00FF
:0E093A00758C009063C012091F120902D2A929
:03094800D28C222C
:0E094B00C0E0C0F0C082C083C002C003C00480
:0E095900C005C006C007C000C001C0D075D0E8
:0A09670000120902120A8C740A251E
:0509710023F523E4352D
:0509760024F524E43526
:05097B0025F525E4351F
:0409800026F526052D
:0609840027E4B52702057F
:01098A002844
:09098B00E527B46404E5286002CC
:02099400800BD6
:080996001208E412115AE4F505
:03099E0027F52812
:0E09A100D0D0D001D000D007D006D005D004B1
:0D09AF00D003D002D083D082D0F0D0E0324F
:05021D00E4F51EF51FD1
:0409BC00AA827B8010
:0C09C0005380EFEB5A6005438008800371
:0309CC005380F75E
:0E09CF00438010EBC313FC8C0370E6438008DA
:0109DD0022F7
:0709DE007A007B805380F7D3
:0B09E5005380EFE58030E203EB42029C
:0E09F000438010EBC313FC8C0370EA438008B5
:0309FE008A8222C8
:0E0A010090E670E0FA54E3F090E670E0FA54EC
:0E0A0F00FDF053B2F943B2181208F77A007BDB
:010A1D0000D8
:0E0A1E00C3EA9408EB64809480502874284A40
:0E0A2C00FC8B058C82C002C0031209BCD003F3
:0E0A3A00D00275820CC002C0031209BCD003AA
:090A4800D0020ABA00D00B80CDE7
:0E0A51007582011209BC7582381209BC7582CB
:0A0A5F00381209BC7582801209BC30
:0E0A6900E58020E1FB7582381209BC7582A081
:030A77001209BCA5
:0E0A7A00E58020E1FB90E670E0FA4402F0D245
:040A88008AD2AA2242
:0C0A8C007582381209BC7582260209BC74
:0C0A98007582381209BC7582020209BC8C
:0E0AA400C0E0C0F0C082C083C002C003C00426
:0E0AB200C005C006C007C000C001C0D075D08E
:0C0AC00000120A98E5AA30E103020BE2E4
:0B0ACC00AA2690F000EAF0000000AA4B
:0A0AD7002590F001EAF0000000AAEB
:0C0AE1002490F002EAF00000007A047B90
:0C0AED0000AC237D007E007F0090F00331
:090AF900ECF00000007C007D001F
:0E0B0200C3EC9408ED648094804003020BCC99
:0E0B100074484CFE8D078E82C002C003C004E4
:0E0B1E00C0051209BCD005D004D003D0028A55
:080B2C00068B070ABA00010B59
:0E0B340074F02FFFC002C003C004C005C0064D
:0E0B4200C0071209DEA882D007D006D005D069
:0E0B500004D003D0028E828F83E8F0000000F4
:090B5E008A068B070ABA00010B9C
:0E0B670074F02FFFC002C003C004C005C0061A
:0E0B7500C0071209DEA882D007D006D005D036
:0E0B830004D003D0028E828F83E8F0000000C1
:090B91008A068B070ABA00010B69
:0E0B9A0074F02FFFC002C003C004C005C006E7
:0E0BA800C0071209DEA882D007D006D005D003
:0E0BB60004D003D0028E828F83E8F00000008E
:050BC4000CBC00010D56
:030BC900020B021A
:0E0BCC008A048B0590E690EDF00000007B009F
:080BDA0090E691EAF000000032
:070BE200051EE4B51E02052B
:010BE9001FEC
:090BEA00E51EB46404E51F60027D
:020BF300800878
:070BF5001208F7E4F51EF5FC
:010BFC001FD9
:0E0BFD00D0D0D001D000D007D006D005D00453
:0D0C0B00D003D002D083D082D0F0D0E032F0
:07022200756900756A0075A3
:060229006400E4F565F538
:04022F0066F567F514
:010233006862
:080C180085827385837485F069
:050C200075E4F57AF512
:040C25007BF57CF5EA
:040C29007DF576F5EA
:040C2D0077F578F5EA
:040C310079AD6EAE7D
:040C35006FAF7085A8
:030C3900717E8544
:020C3C00727FC5
:050C3E00A87EAA7F154D
:070C43007E74FFB57E02156F
:010C4A007F2A
:0E0C4B00C3E49874808AF063F08095F0504105
:0E0C59008D828E838FF01214CCFAA3AD82AE82
:0A0C670083E4FBFCF8EA2576F5763D
:070C7100EB3577F577EC3558
:050C780078F578E83575
:040C7D0079F579E5A7
:040C810076257AF565
:040C85007AE5773560
:040C89007BF57BE597
:040C8D0078357CF545
:040C91007CE5793550
:050C95007DF57D80A447
:0A0C9A00AA767B007C007D008573C4
:090CA400828574838575F0EA1263
:050CAD001326AA6BAB49
:040CB2006CAC6DAD0C
:0C0CB6007A7E007F0078008A828B838C9D
:050CC200F0ED02132615
:0A0CC700AA82AB83ACF0AD6BAE6CFB
:090CD1008D078E001DBDFF011E00
:0E0CDA00C3E49F748088F063F08095F0501F93
:0E0CE8008A828B838CF01214CCF5C1A3AA82F1
:060CF600AB837FA8780229
:050CFC001FBFFF0118FD
:060D0100EF4870F780CA04
:010D070022C9
:070D08007529B5752A62751B
:060D0F002B06752C08758F
:060D15002D06752E00758D
:060D1B002FFA753000758F
:060D21003101753200757E
:060D270033007534007575
:030D2D006B3675AD
:060D30006C00756D4075BA
:030D36006E2B75AC
:060D39006F0075704075AB
:060D3F00710AE4F5729058
:090D4500003575F040120C187520
:060D4E006B0EE4F56C9051
:080D5400002975F040020CC7F4
:070D5C007537B575386275AB
:060D63003906753A077520
:060D69003B14753C00750F
:060D6F003D40753E427597
:060D75003F0F7540007500
:060D7B0041E8754203751A
:060D8100430075440075FB
:060D8700450175460075F0
:060D8D00470075480075E7
:060D93004932754A0075AB
:060D99004B34754C03759C
:060D9F004D00754E0075C9
:060DA5004F0075500075BF
:030DAB006B527513
:060DAE006C00756D40753C
:030DB4006E397520
:060DB7006F00757040752D
:060DBD007118E4F57290CC
:090DC300005175F040120C187586
:060DCC006B1CE4F56C90C5
:080DD200003775F040020CC768
:090DDA00AA827556B575576275C1
:060DE30058067559017568
:060DE9005A06755B008A4A
:030DEF005C8553CD
:050DF2005D755E008547
:030DF700545F85C1
:030DFA00556075CC
:040DFD006100756BB1
:050E010063756C007533
:040E06006D40756E58
:050E0A0058756F007532
:070E0F00704075710AE4F563
:080E16007290006275F04012B9
:070E1E000C18756B0EE4F5E2
:080E25006C90005675F04002CC
:020E2D000CC7F0
:0E0E2F0075CDFF75CBFF75CCD975CAD975C8C6
:0E0E3D0034439853D2DF758DB2758BB2438E5D
:0D0E4B001053890F438920D28E43C05312EB
:060E58000D08120D5C758F
:060E5E00530175540075FC
:090E64005500758201120DDA75CA
:060E6D00531175540075DD
:090E73005500758201120DDA75BB
:060E7C00532075540075BF
:090E82005500758201120DDA75AC
:060E8B00532175540075AF
:090E91005500758201120DDA759D
:060E9A005322755400759F
:090EA0005500758201120DDA758E
:060EA900531075540075A2
:0C0EAF005501758202120DDA53B2FE905C
:0E0EBB00E670E0FA4401F0D288D2BCD2ACD28C
:020EC900A8225D
:0E0ECB00C0E0C0F0C082C083C002C003C004FB
:0E0ED900C005C006C007C000C001C0D075D063
:090EE700001208E4E56460527594
:060EF0006BE8756C037550
:060EF6006D00756E008521
:060EFC0065828566838516
:050F020067F0E5681234
:0E0F070013ADAA82AB83ACF0FD0ABA00090B51
:080F1500BB00050CBC00010D3E
:070F1D00756BE8756C0375AC
:0A0F24006D00756E008A828B838CCD
:0A0F2E00F0ED12133F858223858346
:050F38002485F025F501
:040F3D0026756400B1
:0E0F4100D0D0D001D000D007D006D005D0040B
:0D0F4F00D003D002D083D082D0F0D0E032A9
:0E0F5C00C0E0C0F0C082C083C002C003C00469
:0E0F6A00C005C006C007C000C001C0D075D0D1
:060F780000109902800048
:060F7E002098030210960A
:0B0F8400AA99C298BAB506756A01026E
:020F8F001060F0
:070F9100E56A700302106025
:070F9800E56AB40102800EBE
:070F9F00E56AB402028018AC
:070FA600E56AB40334802268
:0A0FAD00BA62077401256AFB800296
:020FB7007B00BD
:050FB9008B6A021060CC
:0A0FBE00BA02077401256AFB8002E5
:020FC8007B00AC
:050FCA008B6A021060BB
:050FCF00BA10028006CB
:060FD400756A00021060C6
:050FDA00056A02106031
:080FDF00056AE56AB40703028C
:020FE7001055A3
:070FE900E56AB40802800C68
:070FF000E56AB40902800567
:050FF700E56AB40A6484
:0C0FFC008A037C007D007E00AF6A780054
:0E100800EF24F9FFE834FFF8C40354F8CFC416
:0E10160003CF6FCF54F8CF6FF88FF005F08046
:011024000CBF
:0C102500EB2BFBEC33FCED33FDEE33FE57
:0A103100D5F0F1EB2565F565EC350F
:05103B0066F566ED35CD
:0510400067F567EE35C5
:0410450068F568E5FD
:081049006AB40A137564017515
:041051006A00800BA6
:061055008A657566007556
:05105B0067007568004C
:0A106000E5AA20E32EAB6905698BB9
:0C106A00827583F4EAF0000000E569B430
:0C107600401EAA697B0090E694EBF0009D
:0D10820000007B0090E695EAF0000000758C
:04108F006900800371
:031093001208E45C
:0E109600D0D0D001D000D007D006D005D004B5
:0D10A400D003D002D083D082D0F0D0E03253
:0A10B100C0D075D00010C10280000D
:0510BB00A2C0D0D032FC
:0E10C00090E601E0FA54FDF043B3835390FE36
:0710CE0043900253907F22C2
:0E10D500AA827B047C007D087E007F00439091
:0D10E300015390FD43B38043908043900281
:0C10F0005390FDEB5A6005439080800394
:0310FC0053907F8F
:0E10FF00439002EBC313F8880370E653907C15
:0E110D004390025390FD4390025390FD439097
:07111B00025390FD53B37F66
:0B112200E59030E706EC4206ED4207C6
:0E112D004390025390FD8C02EDC313CA13CA07
:0E113B00FB8A048B05EA4B70DE4390028E8225
:031149008F83226F
:0E114C0090E671E0FA54EFF043B4100210C0C8
:08115A00E5AA30E303021207CD
:0B116200AA2690F400EAF0000000AAAA
:0A116D002590F401EAF0000000AA4A
:0C1177002490F402EAF00000007A047BEF
:0C11830000AC237D007E007F0090F40390
:09118F00ECF00000007C007D0082
:0E119800C3EC9403ED64809480504E8C82C0B2
:0E11A60002C003C004C0051210D5AE82AF8394
:0E11B400D005D004D003D0028A008B010ABA05
:0311C20000010B1E
:0E11C500888274F429F5838F00E8F0000000A2
:0911D3008A008B010ABA00010B2D
:0E11DC00888274F429F5837F00EEF000000095
:0711EA000CBC00AA0D80A758
:0E11F1008A048B0590E694EDF00000007B0070
:0811FF0090E695EAF000000003
:0712070043A01053A0EF22E9
:0E120E001201000200000040B40404100100B0
:04121C0001020001CA
:0A1220000A06000200000040010071
:0E122A000902200001010080320904000002C8
:0E123800FF0000000705820200020007058487
:0412460002000200A0
:0E124A000902200001010080320904000002A8
:0E125800FF0000000705820240000007058429
:041266000240000042
:04126A00040309046C
:0E126E001003430079007000720065007300E9
:02127C007300FD
:0E127E000E0345005A002D005500530042009B
:02128C00000060
:03004300021A009E
:03005300021A008E
:091A00000207C4000207DC000229
:081A090007F2000208080002C8
:081A1100082000020862000237
:081A190008AC000208AD000258
:081A210008AE000208AF00024C
:081A290008B0000208B1000240
:081A310008B2000208B3000234
:081A390008B4000208B5000228
:081A410008B6000208AD000226
:081A490008B7000208B8000212
:081A510008B9000208BA000206
:081A590008BB000208BC0002FA
:081A610008BD000208AD0002FF
:081A690008AD000208AD000207
:081A710008BE000208BF0002DC
:081A790008C0000208C10002D0
:081A810008C2000208C30002C4
:081A890008C4000208C50002B8
:081A910008C6000208C70002AC
:081A990008C8000208C90002A0
:081AA10008CA000208CB000294
:081AA90008CC000208CD000288
:071AB10008CE000208CF007F
:08128E00FB7A20E4FCFDFEFFE9
:0E129600E5822582F582E58333F583E5F033AA
:0B12A400F5F0EB33FB4017DAE9804265
:0E12AF00E5822582F582E58333F583E5F03391
:0512BD00F5F0EB33FB2E
:0E12C200EC33FCED33FDEE33FEEF33FFEC9525
:0612D0006BED956CEE953C
:0812D6006DEF956E4013EC95DD
:0812DE006BFCED956CFDEE9533
:0912E6006DFEEF956EFF438201DD
:0212EF00DABE65
:0212F100EB22EE
:0C12F30030040A90E680E0FA440AF08023
:0112FF0008E6
:0813000090E680E0FA4408F0D9
:0D1308009005DC12144A90E65D74FFF09031
:0E131500E65F74FFF05391EF90E680E0FA542B
:03132300F7F022BE
:0601E500E478FFF6D8FDEE
:0801C3007900E94400601B7A99
:0501CB0000901507780B
:0301D0000075A017
:0A01D30000E493F2A308B80002054F
:0801DD00A0D9F4DAF275A0FFCD
:0E13260020F71030F6118883A88220F507F614
:05133400A88375830091
:011339002291
:03133A00F280F747
:02133D00F0229C
:0C133F00AAF0FBE582856BF0A4FCADF089
:0C134B00E583856BF0A42DFDE435F0FE79
:0C135700E582856CF0A42DFDE5F03EFE63
:0C136300E433FFEA856BF0A42EFEE5F0F9
:0C136F003FFFE583856CF0A42EFEE5F046
:0C137B003FFFE582856DF0A42EFEE5F03A
:0B1387003FFFEB856BF0A42FFFEA8511
:0A1392006CF0A42FFFE583856DF0D9
:0C139C00A42FFFE582856EF0A42F8EF0D8
:0513A8008D838C822200
:0801EB007800E84400600A7985
:0301F3000075A0F4
:0601F60000E4F309D8FC4F
:0801FC007800E84400600C7972
:0B02040000900000E4F0A3D8FCD9FA41
:0E13AD00FBC2D530E715D2D5E4C39582F58298
:0D13BB00E49583F583E495F0F5F0E49BFBE9
:0A13C800E56E30E717B2D5E4C395D7
:0513D2006BF56BE495D2
:0513D7006CF56CE495CB
:0513DC006DF56DE495C4
:0313E1006EF56E38
:0E13E400EB12128E30D513FBE4C39582F58216
:0C13F200E49583F583E495F0F5F0E49BAE
:0113FE0022CC
:0613FF00AA82AB14AC153C
:0E1405008B828C83A3E0FDBD03238A051AEDC4
:0714130070058B828C83221F
:0E141A008B058C068B828C83E0FF7800EF2D13
:0A142800FDE83EFE8D038E0480D324
:041432009000002204
:0E14360090E682E044C0F090E681F04387012A
:0614440000000000002280
:0E144A00AA82AB8390E600E0FC541870117487
:0E145800012AFCE43BFD8C02C313CA13CAFB3D
:021466008012F2
:0E14680090E600E0FC530418BC1007EBCA2508
:04147600E0CA33FB9A
:09147A008A048B051ABAFF011B5C
:0E148300EC4D600DC002C0031214E8D003D07F
:031491000280E6F0
:011494002235
:0E14950090E682E0FA30E00890E682E0FA206D
:0214A300E61051
:0E14A50090E682E0FA30E11E90E682E0FA3036
:0214B300E7163A
:0E14B50090E680E0FA4401F090001412144A10
:0814C30090E680E0FA54FEF00F
:0114CB0022FE
:0301B60075817FD1
:0A01B9001214F9E582600302023718
:0E14CC0020F71430F6148883A88220F507E676
:0614DA00A88375830022C7
:0314E000E280F7B0
:0314E300E493226D
:0214E600E02202
:0914E8007400F58690FDA57C0559
:0814F100A3E582458370F92296
:0414F90075820022D6
:00000001FF
